:100000000C94B5010C94ED010C94ED010C94ED01F0
:100010000C94ED010C94ED010C94ED010C94ED01A8
:100020000C94ED010C94ED010C942B1B0C94FD1B16
:100030000C9428160C94ED010C94ED010C94ED0138
:100040000C94ED010C94ED010C94ED010C94ED0178
:100050000C94ED010C94B0160C94ED010C94ED0190
:100060000C94ED010C94ED010C94ED010C94ED0158
:100070000C94ED010C94ED010C94ED010C94ED0148
:100080000C94ED010C94ED010C94ED010C94ED0138
:100090000C94ED010C94ED010C94ED010C94ED0128
:1000A0000C94ED010C94ED010C94ED018C048C0486
:1000B000B804B80420054B064B064B063E05D70591
:1000C000E805E8056A1C911C891D911C891DDD1C31
:1000D000001D891D571D661D3A003B0029001E00AA
:1000E0001F002000210022002300240025002600FC
:1000F00027002D002E002A004A003C003D002B0066
:1001000014001A000800150017001C0018000C004D
:10011000120013002F00300031004B003E003F0062
:10012000390004001600070009000A000B000D004A
:100130000E000F0033003400280000004E00400085
:100140004100E10000001D001B0006001900050031
:1001500011001000360037003800E50052004D0055
:1001600042004300E000E300E20000000000000065
:100170002C00000000000000000001515000510060
:100180004F000100010035003A003B003C003D00FB
:100190003E003F0040004100420043004400450053
:1001A0004C000100010001000100010001000100FC
:1001B0000100010001000100460047004800010065
:1001C000010001000100010001000100AA00A900D6
:1001D000A800B000010001000100010001004A0078
:1001E0000100010000000100010001000100000009
:1001F00001000100010001000100010001000100F7
:1002000001000100010001000100010001000100E6
:1002100001000100000000000000010000000000DB
:10022000000000000100010001000100260377002A
:1002300069006C00620061002E00740065006300BC
:100240006800200057005400360035002D0058008B
:10025000540000001603770069006C006200610022
:100260002E007400650063006800000004030904A8
:1002700009023B00020100A0FA0904000001030189
:100280000100092111010001224000070581030836
:10029000000109040100010300000009211101000F
:1002A00001226D00070582032000011201000200F7
:1002B00000000882651D000100010200010501091E
:1002C00080A101850319012AB700150126B7009501
:1002D0000175108100C0050C0901A10185041901F7
:1002E0002AA002150126A002950175108100C00503
:1002F000010906A1018506050719E029E715002572
:10030000019508750181020507190029EF150025DF
:100310000195F075018102050819012905950575FA
:10032000019102950175039101C005010906A10122
:10033000050719E029E715002501950875018102D7
:100340009501750881010507190029FF150026FF91
:1003500000950675088100050819012905950575A0
:10036000019102950175039101C011241FBECFEFC9
:10037000DAE0DEBFCDBF04B603FE18C08091D5021F
:100380009091D602A091D702B091D8028730904BBD
:10039000A740B04B59F41092D5021092D602109299
:1003A000D7021092D802E0E0F8E3099511E0A0E04E
:1003B000B1E0E8E2FCE302C005900D92AA38B10773
:1003C000D9F722E0AAE8B1E001C01D92A53DB2072D
:1003D000E1F70E9486120C94121E0C94000081E03A
:1003E000089581E008950C94F10108950C94F501AD
:1003F0001F93CF93DF9300D000D01F92CDB7DEB70D
:1004000049835A836B8330918D0189819A8131119F
:1004100014C0662359F0222349F00E948408182F43
:10042000682F89819A810E942D0803C00E94580874
:10043000182F69817A81812F04C00E948408698104
:100440007A810F900F900F900F900F90DF91CF91C6
:100450001F910C94D00FFC01262F408151816281A5
:10046000738184810C94F80181E00895CF93DF9328
:10047000EC0160E00E942B02BE01DF91CF910C9451
:10048000F6010C9419110C94151108950E94D706C9
:100490000E9445022FEF84E39CE021508040904071
:1004A000E1F700C000000C94D6160F931F93CF9372
:1004B000DF938C0161E00E942B02EC01B8010E94E5
:1004C000F3018823F1F1B801CE010E947F14882343
:1004D000C1F1B801CE010E949312882391F1B801B5
:1004E000CE010E94DB13882361F1F8018281882309
:1004F00009F1CB358DE5D807C1F050F4C115FCE505
:10050000DF0781F0CF3DDC45A9F40E94BB0D19C087
:10051000CC35EDE5DE0761F0CD35DD4559F40E94BF
:10052000FE0C08C00E9446020CC00E94070D02C0CB
:100530000E940A0DC801DF91CF911F910F910C9479
:10054000EF0180E0DF91CF911F910F9108950E94FC
:1005500008160C94C0020E94C3020C940E16089553
:100560000C94AF0281E008950C94B2020895CF93E9
:10057000C82F0E94B0028C2F0E94B402CF91089520
:1005800080E00C94B7020E94DB140C94B7020E9426
:10059000DB1490918C01891721F080938C010C94CD
:1005A000B7020895CF93DF93CDB7DEB72B970FB681
:1005B000F894DEBF0FBECDBF4F83588769877A8717
:1005C0008B8761110E944A0C9E012F5F3F4F86E08E
:1005D000F90111928A95E9F785E0FE013796D90174
:1005E00001900D928A95E1F789819A814C815D8114
:1005F000452B31F09F3F31F491E08F3F19F403C058
:1006000091E001C090E090FF09C049815A816B815F
:100610007C818D819E810E946B0B05C0C9010E9467
:1006200034028111F2CF2B960FB6F894DEBF0FBEC5
:10063000CDBFDF91CF910895FC01808191810E940F
:10064000C6080895CF93882309F49CC0C82F823828
:10065000C1F40E94DB1481FD95C069E38091020121
:10066000909103010E94C3150E946C0C2FEF81EE44
:1006700094E0215080409040E1F700C0000069E321
:1006800019C0833801F50E94DB1480FD7BC063E54F
:1006900080910201909103010E94C3150E946C0C8D
:1006A0002FEF81EE94E0215080409040E1F700C0B0
:1006B000000063E580910201909103010E94CE1534
:1006C000CF910C946C0C8438C1F40E94DB1482FD31
:1006D00059C067E480910201909103010E94C31503
:1006E0000E946C0C2FEF81EE94E0215080409040EE
:1006F000E1F700C0000067E4DDCF8CEF8C0F813A9A
:10070000D0F46C2F80910201909103010E94431557
:10071000882349F06C2F80910201909103010E947F
:10072000CE150E946C0C6C2F8091020190910301F8
:100730000E94C315C5CF80E28C0F883048F4C77083
:1007400081E001C0880FCA95EAF70E942D0CB8CF4E
:10075000EBE5EC0FE33040F4F0E0E15CFE4F80812C
:1007600090E0CF910C940115C85AC73158F4EC2F82
:10077000F0E0EE0FFF1FEF5EFE4F80819181CF9181
:100780000C941715CF910895882309F45BC0682F46
:10079000823879F40E94DB1481FF54C069E38091B0
:1007A0000201909103010E94C3150E946C0C69E341
:1007B00010C08338B1F40E94DB1480FF43C063E5AE
:1007C00080910201909103010E94C3150E946C0C5C
:1007D00063E580910201909103010E94CE150C9473
:1007E0006C0C843879F40E94DB1482FF2BC067E420
:1007F00080910201909103010E94C3150E946C0C2C
:1008000067E4E7CF8CEF860F813A18F380E2860F1A
:10081000883048F4677081E001C0880F6A95EAF774
:100820000E94330CDCCF8BE5860F833020F480E010
:1008300090E00C940115685A673120F480E090E054
:100840000C94171508951F93CF93DF93182FEB0186
:100850000E942203209741F08FE99FE00197F1F772
:1008600000C000002197F6CF812FDF91CF911F911B
:100870000C94C403893319F060E070E002C060E5B5
:1008800070E00C942304882321F00E942D0C0C941A
:100890006C0C0895882321F00E94330C0C946C0C8E
:1008A0000895CF92DF92EF92FF920F931F93CF9311
:1008B000DF937C01D62FC72FFC01128105810295A1
:1008C0000F700E94230C8823B9F01123A9F08C2FFC
:1008D000807F803421F080E28D0F883068F0809135
:1008E0009B0282FD09C082E00E94CC0C0E94230C76
:1008F00091E0D82ED92601C0D12CCC2EC2948FE005
:10090000C8228C2D90E08C30910508F0C4C1FC0108
:10091000EA5AFF4F0C94BD1D8C2F807FCF70882327
:1009200011F0C295C07F112399F0CC2309F49FC127
:1009300080E28D0F883010F0D11104C08C2F0E94FE
:100940002D0C03C08C2F0E943D0C0E946C0C8FC19B
:100950008D2F0E94C403CC2309F49DC180E28D0F2A
:10096000883038F1DD2329F18C2F0E94430C24C0FC
:100970008C2F807FCF70803211F0C295C07FDD2335
:1009800019F0D130A1F13DC080919B0282FF17C0C8
:10099000112349F0CC2329F08C2F0E942D0C0E94AA
:1009A0006C0C80E065C180E00E94C403CC2309F494
:1009B00072C18C2F0E94330C0E946C0C6CC11123ED
:1009C00071F0002341F0013031F40E944D0C8C2B6A
:1009D0000E94550C60C10E944D0C8C2B1DC0002341
:1009E00019F0013009F457C10E94620C25C011238F
:1009F00021F0063008F04FC10EC0053008F04BC1A1
:100A00001BC0112361F0002331F0F701858180FFC5
:100A10002EC18F7085838C2F0E9443043CC100231C
:100A200059F0D93309F034C1FFEF07EE13E0F1506C
:100A300000401040E1F72AC18C2F0E944A042BC1CC
:100A40008C2F86958695837019F0813061F023C1D3
:100A5000112321F08D2F9C2F937002C080E090E035
:100A60000E94011520C1112321F08D2F9C2F93701E
:100A700002C080E090E00E94171515C18C2F837092
:100A800009F047C011110BC12D2F22952695277013
:100A9000220F220F6D2F6F70862F90E0A0E0B0E044
:100AA000022E04C0880F991FAA1FBB1F0A94D2F7F9
:100AB000D4FF10C04FE050E060E070E004C0440F8D
:100AC000551F661F771F2A95D2F740955095609560
:100AD000709503C040E050E0BA01C695C695C3705A
:100AE0008A019B01082B192B2A2B3B2BC901B8012A
:100AF000C23049F058F4C13019F00E944307CFC00A
:100B00000E943107CCC00E945507C9C00E942F0720
:100B1000C6C0112319F08C2F817001C086958823DF
:100B200009F4BDC02D2F229526952770220F220F84
:100B30006D2F6F70862F90E0A0E0B0E0022E04C011
:100B4000880F991FAA1FBB1F0A94D2F7D4FF10C0A9
:100B50004FE050E060E070E004C0440F551F661F96
:100B6000771F2A95D2F7409550956095709503C0F0
:100B700040E050E0BA01C695C695C3708A019B015A
:100B8000082B192B2A2B3B2BC901B801C23049F085
:100B900058F4C13019F00E94080881C00E94F6077D
:100BA0007EC00E941A087BC00E94690778C0CF707F
:100BB000112339F08C2F0E948F078D2F0E94430440
:100BC0006EC08D2F0E944A048C2F0E94B00767C010
:100BD000D23F21F128F4D03F41F0D13FC1F043C0D2
:100BE000D33F19F1D43F79F03EC0112341F00530D5
:100BF00008F051C08C2F8F710E94D5074CC0063071
:100C000008F049C0F7CF80919B0282FF18C01123E2
:100C100039F08C2F8F710E948F073DC01123C9F3CB
:100C20008C2F8F710E94B00736C0112329F08C2FB2
:100C30008F710E947A072FC00E9475072CC0112364
:100C400049F0CF718C2F0E948F0763E08C2F0E9498
:100C5000B10C21C081E00E94CC0C0230E0F082E0B7
:100C60000E94CC0C18C0112331F0002391F28D2F7B
:100C70000E94220310C0002399F2D93349F41FEFD8
:100C800027EE33E0115020403040E1F700C0000073
:100C90008D2F0E94C40388EF8C0D843020F40E94B5
:100CA000DB140E94B702DD20C9F00E941F0C80FDFA
:100CB00015C0F70112820E94190C0E948F07C7010C
:100CC0000E948F060E94190CDF91CF911F910F9106
:100CD000FF90EF90DF90CF900C94B007DF91CF9111
:100CE0001F910F91FF90EF90DF90CF9008950F9399
:100CF0001F93CF93DF93EC01688179818A810E94F1
:100D0000D1088C010E942C080E941D07B801CE0159
:100D10000E945104DF91CF911F910F910895CF93BD
:100D2000DF93EC01988189812B813C81232B31F069
:100D30008F3F31F481E09F3F19F403C081E001C08F
:100D400080E080FD1DC0CE010E945502811110C0BF
:100D50000E94230C8823A1F08A81882389F0809146
:100D60009B0282FD0DC082E0DF91CF910C94CC0CF0
:100D7000CE010E947706CE01DF91CF910C9436020E
:100D8000DF91CF91089580E090E00E94011580E00E
:100D900090E00E9417150E944A0C0C946C0C8091F4
:100DA0000201909103010E94D9150C94C3060E9480
:100DB0003A0C0C94CF0692959F70963079F010F40F
:100DC000925001C09A50923068F4803F69F018F454
:100DD000883E40F409C0843F29F406C0883E20F0D4
:100DE000813F11F080E0089581E00895FC01808149
:100DF00091810E94C6080E94DB060895CF93DF937D
:100E000000D000D01F92CDB7DEB70F900F900F909B
:100E10000F900F90DF91CF910895CF93DF9300D083
:100E200000D000D0CDB7DEB726960FB6F894DEBF5F
:100E30000FBECDBFDF91CF910895089508950C9412
:100E40001E070C941F070E9421076093C90170932D
:100E5000CA018093CB019093CC010C94C3060C94EF
:100E600023070F931F930091C9011091CA0120918C
:100E7000CB013091CC01602B712B822B932B1F91D6
:100E80000F910C9423070F931F930091C9011091A8
:100E9000CA012091CB013091CC01602371238223C0
:100EA00093231F910F910C9423070F931F9300918D
:100EB000C9011091CA012091CB013091CC0160276A
:100EC0007127822793271F910F910C9423070C946D
:100ED0001E070E9467076093C5017093C601809347
:100EE000C7019093C8010C94C30660E070E0CB0189
:100EF0000C9469070F931F9341E050E060E070E0AD
:100F00008A019B0104C0000F111F221F331F8A9505
:100F1000D2F7C901B8011F910F910C9469070F9383
:100F20001F9341E050E060E070E004C0440F551FA3
:100F3000661F771F8A95D2F78091C5019091C601EF
:100F4000A091C701B091C8018A019B01082B192B00
:100F50002A2B3B2BC901B8011F910F910C946907F3
:100F60000F931F9341E050E060E070E004C0440F35
:100F7000551F661F771F8A95D2F74095509560954B
:100F800070958091C5019091C601A091C701B09163
:100F9000C8018A019B01082319232A233B23C90185
:100FA000B8011F910F910C9469070F931F9341E0B3
:100FB00050E060E070E004C0440F551F661F771FCB
:100FC0008A95D2F78091C5019091C601A091C70181
:100FD000B091C8018A019B01082719272A273B27BE
:100FE000C901B8011F910F910C9469070F931F93CA
:100FF0000091C5011091C6012091C7013091C8012F
:10100000602B712B822B932B1F910F910C946907EE
:101010000F931F930091C5011091C6012091C70144
:101020003091C80160237123822393231F910F9174
:101030000C9469070F931F930091C5011091C6018D
:101040002091C7013091C80160277127822793271B
:101050001F910F910C946907089521E1929F800DD3
:101060001124E82FE695E695E695877051E001C0DA
:10107000550F8A95EAF785E0E89FF0011124E257C1
:10108000FE4F20E030E070E04081CB01022E02C034
:10109000969587950A94E2F7817081958427852338
:1010A000842781932F5F3F4F2530310569F70895DD
:1010B00021E1929F800D1124682F669566956695B3
:1010C000982F977085E0689FB001112440E050E0B0
:1010D00080E0FB01E40FF51FE257FE4F208130E076
:1010E000092E02C0369527950A94E2F7217033271E
:1010F000042E01C0220F0A94EAF7822B4F5F5F4F44
:101100004530510531F70895BF92CF92DF92EF92AB
:10111000FF920F931F93CF93DF938C01C090C50173
:10112000D090C601E090C701F090C8018091C9013C
:101130009091CA01A091CB01B091CC01C82AD92AC3
:10114000EA2AFB2ACFE1D0E0D701C6010C2E04C069
:10115000B695A795979587950A94D2F780FD04C018
:10116000219790F7B12C07C0BC2EB8018C2F0E949C
:10117000E30F0197A9F38B2DDF91CF911F910F9171
:10118000FF90EF90DF90CF90BF900895CF93DF93C3
:10119000EC010E948408BE010E94E30FDF91CF9111
:1011A00008951F93CF93DF93EB0190918D019923C5
:1011B00021F0CB010E94C60813C0882349F0CB015F
:1011C0000E948408182F682FCE010E942D0804C0A9
:1011D000CB010E945808182FBE01812F0E94E30FF7
:1011E000DF91CF911F9108951F93CF93DF93C0910B
:1011F000CD0116E08091CE01C81799F0D0E01C9F78
:10120000F0011D9FF00D1124E153FE4F40815181EB
:1012100062817381848195810E940D072196C77038
:10122000E9CFDF91CF911F9108954091FF01509137
:10123000000260910102709102028091030290917C
:1012400004020C940D07EF92FF920F931F93CF931C
:10125000DF938091040282958F7009F065C08091C0
:101260000102882309F460C08091CD01F090CE0185
:101270001091FF010091000260910202709103023F
:1012800091E01F3F09F090E0C0910001D091010171
:10129000292F96E0E92E8F1509F446C061157105D6
:1012A00021F00F3F21F030E003C031E001C0322FC8
:1012B00090E030FD36C0E89EF001E99EF00D11246B
:1012C000DF01A153BE4F11963C911197301329C0F5
:1012D0003C91311326C012963C911297311121C0D6
:1012E00013964D915C911497461B570B4C175D0755
:1012F000C0F4809104028F70806180930402EC52EC
:10130000FE4F80818F70806180838FEF91E00E941B
:101310008F06DF91CF911F910F91FF90EF900C946A
:10132000F40801968770B7CFDF91CF911F910F918D
:10133000FF90EF9008959F92AF92BF92CF92DF926D
:10134000EF92FF920F931F93CF93DF93CDB7DEB74A
:1013500061970FB6F894DEBF0FBECDBF8C0185E05C
:10136000F801DE011D9601900D928A95E1F7D801F2
:101370001296EC909091FF01E09100022091020200
:10138000309103022115310531F0EF3F31F481E056
:101390009F3F19F403C081E001C080E0B82FB17015
:1013A0009B2E80FD47C1D8014C9111965C911197FD
:1013B0001396AD90BC9014978FEFC82E81E0D82E75
:1013C000F0900102B501621B730B20910001309176
:1013D0000101FF2009F4D9C080910402621773074C
:1013E00008F095C0282F207F09F052C05E1313C06B
:1013F000491311C0FE2CE1100EC08F7080618093E4
:1014000004020E941509C6010E948F068091040201
:10141000F80185834DC1AB2831F05F3F31F481E0A5
:101420004F3F19F403C081E001C080E080FD03C09C
:1014300081E08E2502C080E090E0F82FF170FF2E51
:1014400080FF1CC08091CD012091CE0136E0821733
:1014500009F40BC190E0389FF001399FF00D112481
:10146000E153FE4F6181561306C06081461303C0ED
:101470006281E61203C001968770E9CFFE2CEE2050
:1014800009F416C18091040281608093040254C063
:101490005E1306C0491304C0E11002C0F80199C0F0
:1014A000C8010E94F606882361F1EE2051F12091D7
:1014B0000402822F82958F7090E0029774F08091E1
:1014C000FF019091000298878F831986BB86AA86B8
:1014D0002C87CE0107960E948F0686E0F801AFEFB9
:1014E000B1E001900D928A95E1F70E9423090E94D4
:1014F00015090AC05E1711F1C8010E94F606811194
:101500002CC0C8010E948F06FF24F394D1C0282F5D
:10151000207F81F77A2DB98AA88A6E2D89890E9449
:10152000FE068FEF91E00E948F0686E0D6011D92A5
:101530008A95E9F70E941509F12CBAC04913DCCF4E
:10154000E110DACFF8018583C8010E948F0686E09A
:10155000D6011D928A95E9F7ABC0EE2091F2209159
:101560000402822F82958F7090E002970CF4B5CF21
:101570008091FF01909100029A8389831B82BD8232
:10158000AC822E83CE010196A6CF6217730708F0B6
:1015900044C0FE2CEE2009F4B4CF5E1330C04913D2
:1015A0002EC02091040220FD21C0822F82958F70D1
:1015B000482F50E041155105C9F0F80125834F30FF
:1015C000510541F08F5F982F9295907F822F8F70F9
:1015D000892B8583C8010E948F0686E0F801AFEF52
:1015E000B1E001900D928A95E1F73CC086E0F801E8
:1015F000AFEFB1E001900D928A95E1F759C0C801B3
:101600000E94F606811169CF809104028160809367
:101610000402C8010E948F064BC07A2DB98AA88A9D
:101620006E2D89890E94FE0686E0D6011D928A955C
:10163000E9F718C0EE2009F464CFC8010E94F6064D
:10164000F82E882309F45DCF86E0F801AFEFB1E012
:1016500001900D928A95E1F78FEF91E00E941C03B3
:101660000E9423090E94150923C04D875E878D853E
:101670009E850E94C608292F22952F70223028F4BB
:101680009F7039F0811105C00BC0243028F49F7081
:1016900049F4805E883020F0C8010E948F069F2C9C
:1016A000F92C06C0D80115969C91907F91F7F8CF40
:1016B0008F2D61960FB6F894DEBF0FBECDBFDF91C0
:1016C000CF911F910F91FF90EF90DF90CF90BF903F
:1016D000AF909F9008951F93CF93DF93CDB7DEB760
:1016E0002C970FB6F894DEBF0FBECDBF4F8358873F
:1016F00069877A878B879C87CE0107960E949B0912
:101700008823D1F09F8188852A853B85232B31F062
:101710008F3F31F481E09F3F19F403C081E001C0A5
:1017200080E080FD47C04F81588569857A858B852B
:101730009C850E940D073EC086E0FE013796DE01C3
:10174000119601900D928A95E1F7FF81E8856A85EF
:101750007B856115710531F0EF3F31F481E0FF3F8A
:1017600019F403C081E001C080E080FD23C0209116
:10177000CE0130E0C9010196877099274091CD01D3
:1017800050E084179507F1F1F983EA837D836C8338
:1017900096E0929FD001939FB00D1124A153BE4FAC
:1017A000FE01319601900D929A95E1F78093CE015A
:1017B0000E94F40816E08091CD019091CE01891726
:1017C00071F1189FC001112481539E4F0E949B0903
:1017D000882329F1E091CD011E9FF0011124E153EE
:1017E000FE4F4081518162817381848195810E9485
:1017F0000D078091CD0190E0019687709927809325
:10180000CD01D9CF0E94D7061092CE011092CD0102
:10181000EFEFF1E086E0DF011D928A95E9F72C9663
:101820000FB6F894DEBF0FBECDBFDF91CF911F91F1
:1018300008958091250285958595859508958091D7
:1018400025028770089590912502977081E009F430
:1018500080E0089580914802089590914802892B74
:10186000809348020895809590914802892380933F
:101870004802089510924802089590914702892BDA
:101880008093470208958095909147028923809321
:101890004702089510924702089580912602089504
:1018A00008950C94500C0C94510C90919B0292FD55
:1018B00008C090912602981721F0809326020C947C
:1018C000530C089580912602882329F01092260255
:1018D00080E00C94530C0895CF93DF93E0910201C4
:1018E000F0910301809148028083E0910201F09120
:1018F0000301908180914702892B80838091260289
:10190000882381F0E0910201F09103019081892BFD
:10191000808380910201909103010E942D15811115
:101920000E94620CC0910201D091030140E250E09C
:1019300065E072E0CE010E94C31D892B69F080E250
:10194000FE01A5E0B2E001900D928A95E1F7CE018B
:10195000DF91CF910C94E714DF91CF9108950C940F
:10196000500C90919B0292FD10C098E0899F9001CD
:101970001124262B209325020E948F078091250297
:101980008595859585950C94AF0C0C948F071092D6
:10199000250280E00C94AF0C2091250280958223D3
:1019A00080932502982F977099F430E0482F082EE5
:1019B000000C550B2417350759F090919B0292FDAE
:1019C00007C08595859585950E94B0070C94C70C36
:1019D000089590919B0292FB222720F9281769F025
:1019E00080FB92F990939B0280919A0290919B02C6
:1019F0000E94370D82E00C94CC0C089580919B02DC
:101A000082FB882780F991E089270C94E90C81E01A
:101A10000C94E90C80E00C94E90C6FEF7FEF80E010
:101A200090E00C94FC1D80E090E00E94D81D21E025
:101A3000893E9E4F09F020E0822F089582E090E0D9
:101A40000C94D01D83E090E00C94D01DCF9384E0E3
:101A500090E00E94D01DC82F82E290E00E94D01D2D
:101A60002C2F30E0A901582BCA01CF910895CF93B4
:101A7000C92F682F84E090E00E94DE1D6C2F82E267
:101A800090E0CF910C94DE1DAB01BC018FE090E0A3
:101A90000C94F01DAB01BC0183E190E00C94F01DAF
:101AA00060E070E0CB010C944A0D60E070E0CB0187
:101AB0000E94440D0C94500D69EE7EEF80E090E0A2
:101AC0000E94FC1D60E082E090E00E94DE1D60E06C
:101AD00083E090E00E94DE1D1092C9011092CA01BD
:101AE0001092CB011092CC0160E084E090E00E9463
:101AF000DE1D60E082E290E00E94DE1D60E085E095
:101B000090E00E94DE1D60E086E090E00E94DE1D15
:101B10006FEF87E090E00E94DE1D40E050E0BA01E8
:101B200088E090E00E94F01D60E08DE090E00E946F
:101B3000DE1D40E050E0BA0188E190E00E94F01D17
:101B400060E087E190E00E94DE1D40E050E0BA01D5
:101B50008CE190E00E94F01D60E070E080E290E097
:101B60000E94FC1D40E050E0BA0188E190E00E9434
:101B7000F01D0C94550D0C945C0D682F8EE090E0D8
:101B80000C94DE1D0E9495166093610270936202B0
:101B9000809363029093640260935D0270935E028F
:101BA00080935F0290936002089585B7806885BF37
:101BB00085B7806885BF089581E008950C94DC0D99
:101BC00008950C94E00D0C94E00D0C94E30D0C942E
:101BD000E00D0C94E70D0C94E00D0E94D50D8FEBF9
:101BE00090E10E94D1140E94EB0D0C94E90D0E942B
:101BF000E10D0C94E00D0E94D9100C94B6020E94E5
:101C000080160E94DD110E94FB0D0C94E50D2F92B1
:101C10003F924F925F926F927F928F929F92AF927C
:101C2000BF92CF92DF92EF92FF920F931F93CF93C9
:101C3000DF93CDB7DEB72D970FB6F894DEBF0FBE9A
:101C4000CDBF0E94F211282E81110E94C20D89E49D
:101C500092E09D878C8700E010E0302E802F0E945C
:101C6000FD102B013C01EC85FD8581919191A191A5
:101C7000B191FD87EC875301420188269926AA2657
:101C8000BB2681149104A104B104B1F40F5F1F4F6E
:101C90000530110511F78FEF89838A831B820E941B
:101CA00089168160782F9D838C8349815A816B814D
:101CB0008D810E94D20251C08091650281FD0E94F7
:101CC00009111B86C12CD12C7601C394D501C40106
:101CD0008C219D21AE21BF21892B8A2B8B2B91F149
:101CE0000E94DE0D8823D1F0FB85FE833F824C20CD
:101CF0005D206E207F2081E045284628472809F492
:101D000080E088870E9489168160782F9A8789876A
:101D10004E815F8168858A850E94D202000F111F63
:101D2000000F111FF801E75BFD4F80819181A281B7
:101D3000B381C826D926EA26FB26C082D182E28258
:101D4000F3820BC08B858F5F8B87CC0CDD1CEE1C68
:101D5000FF1C813109F0BACF99CF81E0211001C079
:101D600080E02D960FB6F894DEBF0FBECDBFDF9199
:101D7000CF911F910F91FF90EF90DF90CF90BF9088
:101D8000AF909F908F907F906F905F904F903F901B
:101D90002F9008950E94070E0C94C702CF93DF93F3
:101DA0000E94E80FEC01811522E59207E8F5811504
:101DB00031E5930708F0B6C0883E910528F5803ECE
:101DC000910508F0E9C0883A910570F4853A9105CB
:101DD00008F07AC08130910509F473C008F4D9C0C5
:101DE000049708F0D9C0D5C08F3B910508F0D1C049
:101DF000C85AD0E0CC0FDD1FCE5BDE4F0990D881F2
:101E0000C02DCE019464C9C0811540E5940708F047
:101E100069C0811550E4950708F060C09A95811556
:101E20009F4108F4B9C0B5C0811536E5930728F580
:101E3000811545E5940708F092C0811554E5950792
:101E400008F087C0AC0143705527282F26952695AA
:101E5000C115D34508F06CC081E090E002C0880F46
:101E6000991F4A95E2F740E2249F90011124EC016A
:101E7000C22BD32BCE019C6890C081152AE5920716
:101E800080F4811539E5930708F072C0811548E5A3
:101E9000940708F47EC0D82FCC27CE01806F906ABB
:101EA0007CC090568115904208F073C08D2F8F71C1
:101EB0000E947C10DD27D0628F71AE01582BCA01C1
:101EC0006CC081E090E069C0C55AD0E0C059DE4FD7
:101ED0008881C82FD0E0CE0190645FC0DF70CE0152
:101EE000906A5BC074E0969587957A95E1F7282F04
:101EF00023703C2F337081E090E002C0880F991F5F
:101F00003A95E2F79C68AC01522B9A019C2F9F7086
:101F10009695969550E2959FE0011124C9018C2B6E
:101F20009D2B3BC0D82FCC27CE01816F906A35C046
:101F300081E090E002C0880F991F4A95E2F750E2D5
:101F4000259F90011124EC01C22BD32BCE019A685E
:101F500024C0D82FCC27CE01846F906A1EC00E9467
:101F60007C108F7190E0D82FCC27CE01906215C0E5
:101F70008F700E947C1094E0D695C7959A95E1F7F2
:101F8000CF70D0E0DC2FCC27D0699E01282BC9016F
:101F900004C080E090E001C0CE01DF91CF910895B0
:101FA00025E5829FC0011124FC0121E1729FE00D13
:101FB000F11D1124E60FF11DEE0FFF1FE852FF4F38
:101FC0008591949108950E94D00F0E94CE0E08959D
:101FD0008238910569F1B0F48133910509F46DC03F
:101FE00048F48932910509F463C08A32910509F4F5
:101FF00069C008958533910509F455C08933910569
:10200000B9F00895833E910569F138F4803E910559
:10201000B1F0823E910509F10895863E9105A9F13E
:10202000873E9105B9F1843E910509F064C023C053
:1020300020919A0220FD4FC021FD4DC0089580914E
:102040009A0280FD44C080919B0280FF44C0809131
:102050009A0284FD42C083EE4DC080919A0282FFB5
:1020600038C0F5CF80919A0282FD33C080919B02E7
:1020700080FD31C0ECCF80919B0281FF32C0809106
:102080009A0284FD2AC087EE35C080919A0283FFB0
:1020900026C0F5CF80919A0283FD21C080919B02DA
:1020A00081FD1FC0ECCF80919A0285FD1CC01DC030
:1020B00080919A0285FD19C016C080919A0286FD12
:1020C00016C017C080919A0286FD13C010C089E324
:1020D00011C082EE0FC080EE0DC080E00BC086EE16
:1020E00009C084EE07C089E205C085E303C08AE227
:1020F00001C081E390E0089590919A0292FF0DC093
:10210000282F2871283019F4877F846006C0282F73
:102110002471243011F48B7F886093FF0DC0282F29
:102120002871283119F4877E846106C0282F247114
:10213000243111F48B7E886120919B0220FF0DC019
:10214000382F3871383019F4877F816006C0382FF6
:102150003171313011F48E7F886021FF0DC0282F3E
:102160002871283119F4877E816106C0282F2171DA
:10217000213111F48E7E886194FD877E089580E080
:1021800008950C940D0D0E94F2118FE39CE90197C4
:10219000F1F700C000000E94F21180E00E94FD10E3
:1021A00060FF04C00E94C1100C94D61608950C94D0
:1021B000C3100E94130D811102C00E94BB0D0E942A
:1021C0001E0D809365020E94260D90939B028093C2
:1021D0009A020E94D7100E94220D682F70E080E0C2
:1021E00090E00E942F076091C5017091C601809117
:1021F000C7019091C8010C94670724E0829FC00139
:102200001124FC01E055FD4F608171818281938131
:102210000895089580EA8A95F1F7089500C0089519
:102220000C940A1108950C9412110C9413110C942F
:1022300012110C941711F894E82FE295EF70F0E06A
:1022400031A1282F2F7081E090E001C0880F2A95DE
:10225000EAF7982F9095932391A392A1892B82A3BB
:10226000789408950F931F93CF93DF93C4E8D1E040
:1022700089918F3F11F00E941B1181E0C938D80766
:10228000B9F7C3E7D1E004E811E089918F3F11F07D
:102290000E941B110C171D07C1F7DF91CF911F91F1
:1022A0000F9108954F925F926F927F928F929F92BB
:1022B000AF92BF92DF92EF92FF920F931F93CF9353
:1022C000DF938C01C62FD0E0CE018C579E4F7C014E
:1022D000FC0190819F3F09F460C0D62EF894E92F4D
:1022E000E295EF70F0E081A19F7021E030E001C045
:1022F000220F9A95EAF7822B81A382A120952823A9
:1023000022A378940E940E11E3E7F1E024E831E083
:10231000412C512C32014394812C912C54018191F8
:102320008F3F99F0A82FA295AF70B0E090964C9196
:1023300050E08F70BA0102C0759567958A95E2F7F3
:1023400060FD03C0D301C20103C080E090E0DC0166
:10235000882A992AAA2ABB2A440C551C661C771C79
:102360002E173F07E1F6F70180818F3F11F00E94A1
:102370001B1161E081149104A104B10409F460E02F
:102380008D2D0E941011CC0FDD1FCC0FDD1FC00F53
:10239000D11F88829982AA82BB82DF91CF911F913F
:1023A0000F91FF90EF90DF90BF90AF909F908F9034
:1023B0007F906F905F904F9008950E94321184E15A
:1023C000E0EBF2E0DF01982F1D929A95E9F7ECE936
:1023D000F2E0DF011D928A95E9F785E00E943D1247
:1023E0000C944102FF920F931F93CF93DF93CDB7CD
:1023F000DEB764970FB6F894DEBF0FBECDBF8E0177
:102400000F5F1F4F84E1F80111928A95E9F7F12CD3
:102410006F2DC8010E945211F394F5E0FF12F8CF1E
:1024200044E150E0B8018CE992E00E94C31DFF2412
:10243000F394009709F4F12C892B41F084E1F80121
:10244000ACE9B2E001900D928A95E1F72F2D45E0BD
:1024500060EB72E08CE992E00E943E120E9443021F
:102460008F2D64960FB6F894DEBF0FBECDBFDF91FF
:10247000CF911F910F91FF9008950895FF920F93B0
:102480001F93CF93DF93F82ED92F8B01C42F2223D4
:1024900049F081E0809368020E9489169093670258
:1024A00080936602809168028823F1F08091660231
:1024B000909167020E94A1160597B0F0EF2DFD2FB5
:1024C000D80180E090E04C2F50E08417950754F439
:1024D00001911191219131910D931D932D933D9374
:1024E0000196F3CF10926802DF91CF911F910F9167
:1024F000FF9008950E9483180E94FF0D0C948F187E
:102500000E9493180E94CA0E0C94AD180E942716C0
:102510000E946A180E94ED0D0E947A120E94801299
:102520000E94F70DFBCFCF93DF93EC01FB0182817B
:10253000882309F43CC1C430FDE5DF0760F4CB3FDC
:102540009CE5D90788F49E0122503C452431310591
:1025500008F02EC109C0C236EDE5DE0729F0C63A03
:10256000FDE5DF0709F024C10E94260D90939B0230
:1025700080939A02C1318CE5D80709F4C6C008F0EF
:1025800042C0C930ECE5DE0709F49BC000F5C53058
:102590008CE5D80709F485C078F4C330ECE5DE0794
:1025A00009F478C008F07AC0C230DC4509F0F5C003
:1025B00080919A028160EFC0C7309CE5D90709F489
:1025C00078C008F07AC080919A028061E4C0CD3072
:1025D000FCE5DF0709F487C058F4CB309CE5D90748
:1025E00009F479C008F07BC080919A0288606FC0BE
:1025F000CF30FCE5DF0709F480C008F082C080918D
:102600009A02877FC8C0CE3F9CE5D90709F471C004
:1026100000F5C531FCE5DF0709F485C068F4C33176
:102620009CE5D90709F475C008F095C00E94D7064B
:1026300080919A028F77AFC0CC3FFCE5DF07A9F10C
:1026400008F054C0CB3FDC4509F0A7C080919B0245
:1026500040C0C230EDE5DE0709F489C058F4C11569
:102660008DE5D80709F45AC008F069C080919B0233
:1026700082602FC0C236EDE5DE0709F47CC0C63AA1
:10268000FDE5DF0709F481C0C330DD4509F085C0F1
:1026900080E06EC080919A0282607DC080919A0233
:1026A00016C080919A02886076C080919B028260F9
:1026B0004FC080919A0280626EC080919A028064BD
:1026C0006AC00E94D70680919A02806864C08460C4
:1026D00062C081603DC080919A028E7F5CC0809113
:1026E0009A028D7F58C080919A0216C080919B02F9
:1026F00018C080919B028D7F2BC080919A028F7EA3
:102700004AC080919A028F7D46C080919A028F7B49
:1027100042C080919A02877F8B7F3DC080919B024F
:102720008D7F8E7F15C080919A0282FB222720F92F
:1027300091E0922790FB82F990FB83F92CC0809165
:102740009B02982F909591708E7F892B90FB81F939
:1027500080939B0222C00E94D70680919A0287FB39
:10276000222720F991E0922790FB87F914C081E09D
:102770000E94BD0D12C080919A0284FB222720F98D
:1027800091E0922790FB84F906C080919A02982FDD
:10279000909590FB80F980939A0280919A02909193
:1027A0009B020E94370D0E94D70680E001C081E0A5
:1027B000DF91CF910895CF93DF9386319C4541F50A
:1027C000EB010E942A0C982F8A81209102013091FE
:1027D0000301882379F09A7A81E009F480E08093FC
:1027E0006902911102C069E201C065E3C9010E945A
:1027F000C3150AC080916902811102C069E201C05B
:1028000065E3C9010E94CE150E946C0C80E001C0F6
:1028100081E0DF91CF9108950F931F93CF93DF93C2
:10282000C42FD22FFC0182818823C9F040936C020F
:102830000E94891690936B0280936A0280E28C0F4B
:10284000883008F057C0C77081E001C0880FCA9572
:10285000EAF7DF91CF911F910F910C94430480917F
:102860006C02481330C080916A0290916B020E9402
:10287000A116883C910538F510E21D0FCD17B9F06F
:1028800080E28C0F883040F4C77081E001C0880F6F
:10289000CA95EAF70E944A04183028F581E09D2F76
:1028A000977001C0880F9A95EAF70E944304802F21
:1028B0000E943A041830F0F4D77081E001C0880F0C
:1028C000DA95EAF70AC080E28C0F883098F4C77076
:1028D00081E001C0880FCA95EAF7DF91CF911F917F
:1028E0000F910C944A04802FDF91CF911F910F918B
:1028F0000C943A04DF91CF911F910F9108950F939B
:102900009C01CB01243F4CE5340731F188F4293D8B
:10291000FCE53F07D9F02A3D4CE5340779F1283D25
:102920003C45A9F506E221EE41EE68ED7CE52BC0C1
:10293000263FFCE53F07E1F0A8F0273F3C4539F58D
:1029400007E225EE46EE67EF7CE51DC007E225EEC7
:1029500045EE69ED7CE517C006E221EE40EE64EF3E
:102960007CE511C007E225EE44EE65EF7CE50BC087
:1029700006E221EE42EE66EF7CE505C008E221E0CA
:1029800045EE6AED7CE50E940C1480E008C0FC0175
:102990008281882319F010926C0201C081E00F91AE
:1029A000089590938B0180938A0108959093720209
:1029B000809371020895E0917102F0917202309754
:1029C00021F00190F081E02D099480E00895E091DC
:1029D0007102F0917202309799F020911001222338
:1029E00059F020919A0227FF07C0DC012C91119623
:1029F0002C93119726E02C930280F381E02D09940B
:102A0000089520916F02309170022817390771F0F4
:102A10009093700280936F02E0917102F0917202C4
:102A2000309721F00680F781E02D099408952091D8
:102A30006D0230916E022817390771F090936E0283
:102A400080936D02E0917102F0917202309721F053
:102A50000084F185E02D09940895FC01329680915F
:102A60001001882331F080919A0287FF02C09EE115
:102A700001C096E080E0915028F021912223D9F303
:102A80008F5FF9CF0895662351F120911001222321
:102A9000E9F020919A0227FF19C0462F46954695E6
:102AA00046954E31E0F4677021E030E002C0220F1D
:102AB000331F6A95E2F7FC01E40FF11D828190E07B
:102AC0002823392381E0232B69F409C0FC013296C5
:102AD00008962191621729F0E817F907D1F780E0ED
:102AE000089581E008959C01FC0132969FEF80E0FB
:102AF0004191461789F09F3F19F4411101C0982F69
:102B00008F5F8630A9F79F3F39F0F901E90FF11D7A
:102B100097FDFA956283089508959C012A5F3F4FBF
:102B2000FC014281461301C012820196821793076D
:102B3000B9F70895262F2695269526952E3168F407
:102B4000FC01E20FF11D677021E030E001C0220FAF
:102B50006A95EAF78281282B22830895262F2695ED
:102B6000269526952E3170F4FC01E20FF11D677059
:102B700021E030E001C0220F6A95EAF720958281BA
:102B800028232283089520911001222329F02091E7
:102B90009A0227FD0C949A150C947315209110013C
:102BA000222329F020919A0227FD0C94AE150C9453
:102BB0008D1520911001FC013296222331F0809175
:102BC0009A0287FF02C08EE101C086E0DF011D92FC
:102BD0008A95E9F7089508950C94EB1583E08093A6
:102BE00073020C94EC15811102C081E001C082E0F7
:102BF000809373020C94EC150C94F31581E0809390
:102C000073020C94EC150C94FE1508950C940516A3
:102C10000C9406160C9405160C9405160C940516C7
:102C2000CF930E940C160E94F2110E940A16C0E077
:102C30008C2F0E94FD10672B682B692B29F4CF5F26
:102C4000C530B1F780E001C081E0CF9108950895CB
:102C50001F920F920FB60F9211248F939F93AF93F1
:102C6000BF9380917402811113C08091C40290912E
:102C7000C502A091C602B091C7024196A11DB11D27
:102C80008093C4029093C502A093C602B093C7027A
:102C9000BF91AF919F918F910F900FBE0F901F909A
:102CA00018958091CC02843031F10E94A7021092D5
:102CB000740220E488E190E00FB6F894A895809320
:102CC00060000FBE2093600083B7817F846083BF64
:102CD00083B7816083BF7894889583B78E7F83BFE5
:102CE0000FB6F894A8958091600088618093600089
:102CF000109260000FBE08950E94D7060C94AB029C
:102D000082E084BD93E095BD9AEF97BD80936E00FD
:102D100008952FB7F8948091C4029091C502A091B4
:102D2000C602B091C7022FBF08952FB7F8946091E3
:102D3000C4027091C5028091C6029091C7022FBF54
:102D400008959C014FB7F8948091C4029091C502F8
:102D5000A091C602B091C7024FBF821B930B08958A
:102D600078941F920F920FB60F9211248F939F9316
:102D7000AF93BF938091C4029091C502A091C60207
:102D8000B091C7020196A11DB11D8093C40290931A
:102D9000C502A093C602B093C702BF91AF919F91A5
:102DA0008F910F900FBE0F901F90189581E0809328
:102DB000E00080E28093D8001092C9008FE19EE489
:102DC0000197F1F700C0000087E090EBDC018093F1
:102DD000D5029093D602A093D702B093D8029CE07C
:102DE00088E10FB6F894A895809360000FBE909389
:102DF0006000FFCF8091980208950895CF93DF93EC
:102E000020911001222339F020919A0227FF03C05C
:102E100060E222E002C068E021E02093E9002FEFA9
:102E20003091E800215035FD06C035ED3A95F1F7B7
:102E300000002111F5CF2091E80025FF1DC0EC0115
:102E400080911001811105C040E050E068E070E021
:102E500003C070E040E050E0CE010E941F19809155
:102E6000E8008E778093E80080E2FE01A8E7B2E0F8
:102E700001900D928A95E1F7DF91CF9108958093AB
:102E8000750270937702609376028091CC02843051
:102E900001F582E08093E9008FEF9091E800815086
:102EA00095FD06C095ED9A95F1F700008111F5CFDB
:102EB0008091E80085FF0DC040E050E063E070E0E5
:102EC00085E792E00E941F198091E8008E77809339
:102ED000E8000895BC0184E00C943F17BC0183E036
:102EE0000C943F1708958091CB02811109C00E9474
:102EF000B01A0E940D1B8091E20084608093E20072
:102F000008951092CB0208950C9403166091C802A4
:102F100081E0611101C080E00C94EE159091CC022B
:102F200081E0943009F080E06091C8020C94F315C0
:102F300042E061EC81E00E94291A42E261EC82E009
:102F40000E94291A9091CC0281E0943009F080E02F
:102F50006091C8020C94FC158091CE02833009F474
:102F600061C030F4813071F0823009F49AC0089564
:102F70008A3009F486C08B3009F46CC0893009F0BE
:102F8000A8C020C08091CD02813A09F0A2C08091F2
:102F9000E800877F8093E8008091D1029091D2026F
:102FA000892B21F460E288E792E003C060E080E0D2
:102FB00090E070E00E946A198091E8008B7780931E
:102FC000E80008958091CD02813209F082C080919D
:102FD000D1029091D202029708F07BC08091E80064
:102FE000877F8093E8008091E80082FD05C0809192
:102FF000CC028111F8CF6DC02091F3008091F200D6
:1030000090E0922B029731F48091F100813011F021
:10301000863021F48091F100809398028091E8003D
:103020008B7753C08091CD02813A09F052C08091D4
:10303000D1029091D202892B09F04BC08091E80017
:10304000877F8093E8008091E80080FFFCCF80912B
:10305000100136C08091CD028132D9F58091D10224
:103060009091D202892BA9F58091E800877F809307
:10307000E8000E945E1A8091CF02809310010C94A8
:10308000D7068091CD02813221F58091E800877FBB
:103090008093E8000E945E1A8091D002809399028A
:1030A00008958091CD02813AA1F48091E800877F54
:1030B0008093E8008091E80080FFFCCF8091990226
:1030C0008093F1008091E8008E778093E8000C9463
:1030D0005E1A089584B7877F84BF0FB6F894A895C9
:1030E00080916000886180936000109260000FBE44
:1030F00090E080E80FB6F8948093610090936100AF
:103100000FBE0C94FE150E94B01A0E940D1BE2EE39
:10311000F0E080818460808378940C94A21D84E028
:1031200091E00C94D6148091CC028530A9F4809162
:10313000CC02853079F40E9451168091CA0288230E
:10314000B1F30E941016882391F30E9409190E947E
:10315000D706EDCF0C947C16089508950C94B01802
:10316000292F332723303105C9F060F42130310590
:1031700081F02230310509F044C08BE390E020E774
:1031800032E043C021323105E1F02232310549F10C
:1031900038C082E190E02BEA32E037C099278130D5
:1031A000910549F028F0029761F5ECE2F2E005C0E4
:1031B000ECE6F2E002C0E4E5F2E0849190E09F01E9
:1031C00024C06115710541F061307105D1F489E0C9
:1031D00090E02BE932E019C089E090E022E832E08B
:1031E00014C06115710541F06130710551F48DE62F
:1031F00090E02DEB32E009C080E490E02AE233E079
:1032000004C080E090E020E030E0FA0131832083C8
:10321000089580E189BD82E189BD09B400FEFDCF3A
:103220008091D8008F7D8093D8008091E0008260EB
:103230008093E0008091E00081FDFCCF0895CF9263
:10324000DF92EF92FF920F931F93CF93DF93EC01E6
:103250008B017A010E947D1A811133C0E114F104BF
:1032600039F0F70180819181081B190BC80FD91F14
:10327000C12CD12C0115110519F18091E80085FDB3
:1032800016C08091E8008E778093E800E114F10485
:1032900049F0F70180819181C80ED91ED182C08288
:1032A00085E00FC00E947D1A882321F30AC089910E
:1032B0008093F10001501109FFEFCF1ADF0ADACF36
:1032C00080E0DF91CF911F910F91FF90EF90DF9001
:1032D000CF9008952091D3023091D402261737075A
:1032E00048F06115710539F42091E8002E7720939C
:1032F000E80001C0B901FC0120E06115710579F118
:103300008091CC028823F1F18530F1F18091E800C1
:1033100083FD3CC08091E80082FD2EC08091E800D2
:1033200080FFEBCF2091F3008091F20090E0922B90
:103330006115710551F08830910538F42191209381
:10334000F100615071090196F3CF21E0089709F06F
:1033500020E08091E8008E778093E800CECF2111A5
:10336000CFCF0AC08091CC02882361F0853061F014
:103370008091E80083FD0AC08091E80082FFF2CFCF
:1033800080E0089582E0089583E0089581E0089543
:103390002091D3023091D4022617370748F06115E7
:1033A000710539F42091E8002E772093E80001C0E0
:1033B000B901FC0120E06115710591F18091CC0209
:1033C000882309F440C0853009F43FC08091E800AB
:1033D00083FD3DC08091E80082FD2FC08091E80010
:1033E00080FFE9CF2091F3008091F20090E0922BD2
:1033F0006115710559F08830910540F424912093AE
:10340000F1003196615071090196F2CF21E00897E1
:1034100009F020E08091E8008E778093E800CBCF20
:103420002111CCCF0AC08091CC02882361F0853075
:1034300061F08091E80083FD0AC08091E80082FF7E
:10344000F2CF80E0089582E0089583E0089581E05E
:103450000895982F973068F59093E900981739F000
:103460007091EC002091ED005091F00003C0242FEA
:10347000762F50E021FD02C09F5FECCF3091EB0032
:103480003E7F3093EB003091ED003D7F3093ED00B7
:103490003091EB0031603093EB007093EC0020939F
:1034A000ED005093F0002091EE0027FDE5CF80E085
:1034B00008958F708093E90081E008958091CD0296
:1034C00087FF11C08091E80082FD05C08091CC0289
:1034D0008111F8CF11C08091E8008B770BC08091EB
:1034E000CC02882349F08091E80080FFF8CF8091DA
:1034F000E8008E778093E80008952091E4003091F1
:10350000E50095E64091EC00842F817040FF23C0D8
:103510008091E80080FD1DC08091CC02882399F045
:10352000853099F08091EB0085FD11C04091E40059
:103530005091E5002417350729F3915011F09A01B5
:10354000E1CF84E0089582E0089583E0089581E06A
:10355000089580E008954091E80042FFDDCF08958E
:103560000E941E1B0E94261BE0EEF0E0808181601D
:103570008083E8EDF0E080818F77808319BCA7ED30
:10358000B0E08C918E7F8C9380818F7E80831092AF
:10359000CB0208950F931F93CF93DF930E941E1BBE
:1035A0000E94261BC8EDD0E088818F7788838881B0
:1035B0008068888388818F7D888319BC1092CC02B3
:1035C0001092C8021092CA021092C90200EE10E0D6
:1035D000F80180818B7F808388818160888342E0CD
:1035E00060E080E00E94291AE1EEF0E080818E7FA9
:1035F0008083E2EEF0E0808181608083808188605A
:103600008083F80180818E7F8083888180618883B8
:10361000DF91CF911F910F910895E8EDF0E0808147
:103620008F7E8083E7EDF0E080818160808384E09D
:1036300082BF81E08093CB020C94CA1AE8EDF0E0DF
:1036400080818E7F80831092E20008951092DA00CC
:103650001092E10008951F920F920FB60F9211245D
:103660002F933F934F935F936F937F938F939F938A
:10367000AF93BF93EF93FF938091E10082FF0BC064
:103680008091E20082FF07C08091E1008B7F8093F0
:10369000E1000E94A11D8091DA0080FF1FC080918F
:1036A000D80080FF1BC08091DA008E7F8093DA0003
:1036B0008091D90080FF0DC080E189BD82E189BD84
:1036C00009B400FEFDCF81E08093CC020E94731705
:1036D00005C019BC1092CC020E9481178091E100B4
:1036E00080FF19C08091E20080FF15C08091E20048
:1036F0008E7F8093E2008091E20080618093E200FF
:103700008091D80080628093D80019BC85E08093B6
:10371000CC020E9486178091E10084FF30C0809126
:10372000E20084FF2CC080E189BD82E189BD09B43B
:1037300000FEFDCF8091D8008F7D8093D8008091CE
:10374000E1008F7E8093E1008091E2008F7E809384
:10375000E2008091E20081608093E2008091C802E3
:10376000882311F084E007C08091E30087FD02C048
:1037700081E001C083E08093CC020E948E1780918B
:10378000E10083FF29C08091E20083FF25C0809182
:10379000E100877F8093E10082E08093CC02109269
:1037A000C8028091E1008E7F8093E1008091E20069
:1037B0008E7F8093E2008091E20080618093E2003E
:1037C00042E060E080E00E94291A8091F000886069
:1037D0008093F0000E948417FF91EF91BF91AF9109
:1037E0009F918F917F916F915F914F913F912F9119
:1037F0000F900FBE0F901F9018951F920F920FB64B
:103800000F9211242F933F934F935F936F937F9366
:103810008F939F93AF93BF93CF93DF93EF93FF93D8
:10382000C091E900CF708091EC00D82FD17080FD5D
:10383000D0E81092E9008091F000877F8093F0003B
:1038400078940E94411C1092E9008091F0008860F9
:103850008093F000CD2BCF70C093E900FF91EF91E2
:10386000DF91CF91BF91AF919F918F917F916F9198
:103870005F914F913F912F910F900FBE0F901F902E
:1038800018951F93CF93DF93CDB7DEB7AA970FB6E6
:10389000F894DEBF0FBECDBFEDECF2E08091F100F9
:1038A000819322E0E53DF207C9F70E94AC178091B1
:1038B000E80083FF2EC18091CD029091CE02492F66
:1038C00050E04A30510508F024C1FA01EE59FF4F8B
:1038D0000C94BD1D803821F0823809F01AC108C04F
:1038E0008091C9029091CA02992389F082600FC029
:1038F0008091D1028F70873008F00BC18093E9006E
:103900008091EB0085FB882780F91092E900909167
:10391000E800977F9093E8008093F1001092F10007
:10392000D1C0282F2D7F09F0F4C0882319F08230F0
:1039300061F0EFC08091CF02813009F0EAC093308E
:1039400009F080E08093CA022EC08091CF028111DD
:103950002AC08091D1028F702FEF280F263008F0F7
:10396000D8C08093E9002091EB0020FF1CC0933069
:1039700021F48091EB00806214C09091EB00906183
:103980009093EB0021E030E0A90102C0440F551FE5
:103990008A95E2F74093EA001092EA008091EB00EA
:1039A00088608093EB001092E9008091E800877FA7
:1039B0008093E8000E945E1AACC08111AAC01091E9
:1039C000CF021F778091E3008078812B8093E30002
:1039D0008091E800877F8093E8000E945E1A8091C2
:1039E000E80080FFFCCF8091E30080688093E300D3
:1039F000111102C082E001C083E08093CC0289C033
:103A00008058823008F085C08091CF029091D0021A
:103A10008C3D53E0950779F583E08A838AE28983B8
:103A20004FB7F894DE01139620E03EE051E2E32F19
:103A3000F0E050935700E49120FF03C0E295EF704F
:103A40003F5FEF708E2F90E0EA3010F0C79601C014
:103A5000C0968D939D932F5F243149F74FBF80917E
:103A6000E800877F8093E8006AE270E0CE0101966B
:103A70000E946A1916C06091D1027091D202AE0103
:103A80004F5F5F4F0E94AE18BC01892B09F441C003
:103A90009091E800977F9093E80089819A810E9435
:103AA000C8198091E8008B778093E80032C0803895
:103AB00081F58091E800877F8093E8008091C802BB
:103AC0008093F1008091E8008E7772CF811121C040
:103AD0008091CF029091D00299270297D4F48091DF
:103AE000E800877F8093E8008091CF028093C8022E
:103AF0000E945E1A8091C802811106C08091E30085
:103B000087FD02C081E001C084E08093CC020E9466
:103B100098178091E80083FF0AC08091E800877FB2
:103B20008093E8008091EB0080628093EB00AA967E
:103B30000FB6F894DEBF0FBECDBFDF91CF911F91BE
:103B400008950895CF938091CC028823A1F0C0916D
:103B5000E900CF709091EC00892F817090FD80E892
:103B6000C82B1092E9008091E80083FD0E94411C5F
:103B7000CF70C093E900CF910895EE0FFF1F05901D
:103B8000F491E02D0994FB01DC0104C08D910190BA
:103B9000801921F441505040C8F7881B990B0895B3
:103BA000F999FECF92BD81BDF89A992780B5089505
:103BB000A8E1B0E042E050E00C94041E262FF999F1
:103BC000FECF92BD81BDF89A019700B4021639F07C
:103BD0001FBA20BD0FB6F894FA9AF99A0FBE08954D
:103BE0000396272F0E94DF1D0E94DE1D252F0E94B5
:103BF000DF1D242F0C94DF1D0196272F0E94DF1D4F
:103C00000C94DE1DDC01CB01FC01F999FECF06C04E
:103C1000F2BDE1BDF89A319600B40D92415050408A
:083C2000B8F70895F894FFCFF6
:103C2800C8002702FA16FE1672176E176A17FD16D5
:103C380001E200E900EA00B500B600B700CD008354
:103C480001CC008A01920194012102230224022559
:103C580002260227022A02B300B4006F0070008116
:103C68008283E200E900EA00B500B600B700CD00A3
:103C78008301CC008A0192019401210223022402CB
:103C88002502260227022A02B300B4006F00700042
:103C98008182833730F595313233939267663635B2
:0A3CA80034979694F0F1F4F6F7005B
:00000001FF
